:020000020000FC
:10000000BBC4A2C6A1C6A0C69FC69EC69DC69CC6AE
:100010009BC69AC699C698C697C672C695C694C618
:1000200061C692C691C690C68FC629C68DC68CC6BB
:100030008BC68AC60AFA8CA8782909BA0828FFDD77
:100040000DFDC868C94F594DD9DF3C1C1D0FEED5B9
:10005000309B1CC0329B70C0319BC1C00895009181
:100060000901025050F0CBD302E100930901D9D528
:1000700094D1309BF8CF94D50895C1D302E000937A
:100080000901CFD58AD1309BF8CF0895B8D3042D7C
:10009000003029F3309BFACF009109010030A9F01C
:1000A0000130B9F00430C9F00630E1F00830F9F061
:1000B0000A3011F10B3029F10D3041F10E3059F1B8
:1000C000003171F1013191F1089501E000930901CE
:1000D0000895002700930901089505E000930901A0
:1000E000A0D5089507E0009309019BD5089509E084
:1000F0000093090196D508950BE00093090191D56D
:1001000008950CE0009309018CD508950EE000934A
:10011000090187D508950FE00093090182D508955C
:10012000B8D301E1009309017CD50895A4D502E17B
:100130000093090176D5089562D3042D0030F9F1BA
:10014000329BFACF009109010030A9F0013099F0FB
:10015000043099F0063099F0083099F00A3099F09F
:100160000B30B9F00D30D9F00E30F9F0003119F143
:10017000013119F108957AD50895ECD0089507D189
:100180000895F7D0089500911301A8D000931301AA
:1001900008950091120196D00093120108950091E4
:1001A00015019CD0009315010895009114018AD087
:1001B000009314010895B4D008956CD008951FD30E
:1001C00001E000930A01A8D4329BF9CF089517D318
:1001D00001E000930A01A0D4319BF9CF08950FD319
:1001E000042D0030A1F3319BFACF009109010030BA
:1001F000A9F0013099F0043099F0063099F00830F8
:1002000099F00A3099F00B30B9F00D30D9F00E307A
:10021000F9F0003119F1013119F1089522D508954D
:1002200090D00895ACD008959CD00895009113010A
:100230004FD0009313010895009112013DD0009317
:10024000120108950091150143D0009315010895FE
:100250000091140131D000931401089545D0089500
:1002600001D0089500910B01102F12950F701F708F
:10027000093011F0039507C00027153011F01395D0
:1002800002C0002711270F701F701295010F0093F5
:100290000B01089500910B01102F12950F701F7024
:1002A000003011F00A95EFCF09E0103011F01A95E7
:1002B000EACF09E015E0E7CF0B3311F0039508957D
:1002C00000270895003011F00A9508950BE3089572
:1002D000073111F00395089500270895003011F0BB
:1002E0000A95089507E1089500910C01102F1295C9
:1002F0000F701F70123021F0093031F0039509C0E2
:10030000033029F0039505C00027139502C000278C
:1003100011270F701F701295010F00930C010895A3
:1003200000910C01102F12950F701F70003011F00A
:100330000A95EFCF103011F01A95EBCF03E012E0E1
:10034000E8CF2224009101010F3F09F003950093AB
:10035000010108952224009101010030C1F30A95A2
:10036000F6CF00910001033609F0039500930001D8
:100370000895009100010130C9F30A95F7CF00916B
:100380001101093009F003950093110108950091BE
:1003900011010130C9F30A95F7CF0091090100302E
:1003A00019F1013011F1023009F1033001F104308B
:1003B000F9F00530F1F00630E9F00730E1F00830EF
:1003C000D9F00930D1F00A30C9F00B30C1F00C304F
:1003D000B9F00D30B1F00E30A9F00F30A1F00031BE
:1003E00099F0013191F057C111C013C01CC030C049
:1003F00044C054C068C072C086C08FC0A3C0BCC017
:10040000D5C0E9C002C11BC130C13AC159D163D1C5
:1004100008950AE000931001009103018ED106E1D6
:1004200000930D010895032D003069F003E100935E
:100430000D010CE000930E0105E000930F010AE0AE
:1004400000931001089503E000930901EAD3089591
:10045000032D003069F005E000930D0104E10093E5
:100460000E010CE000930F0105E0009310010895C8
:1004700004E000930901D5D30895022D003039F02E
:100480000091020147D10EE000930D010895009103
:10049000010140D101E100930D010895032D0030C9
:1004A00069F003E100930D0105E000930E010FE0F8
:1004B00000930F0102E100931001089506E00093FC
:1004C0000901AFD308950AE00093100100911101D2
:1004D00034D102E100930D01A4D30895032D00301F
:1004E00069F007E100930D0104E100930E0104E1BE
:1004F00000930F0103E100931001089508E00093B9
:1005000009018FD308950AE00093100100910001C2
:1005100014D106E100930D010895032D003069F018
:1005200004E100930D0100E100930E010AE0009345
:100530000F0101E10093100108950AE00093090101
:1005400070D308950AE00093100100930F01022D6B
:10055000003051F00091130135D100930F0110309C
:1005600009F41AE010931001009112012BD10093AD
:100570000D0110930E0108950AE000930D01009300
:100580000E01022D003039F0009112011BD10093B1
:100590000D0110930E010091130114D100930F016E
:1005A000103009F41AE0109310010895032D003063
:1005B00069F008E100930D0108E100930E0100E1EC
:1005C00000930F0101E10093100108950DE00093E5
:1005D000090127D308950AE00093100100930F0149
:1005E000022D003051F000911501ECD000930F0165
:1005F000103009F41AE01093100100911401E2D0B8
:1006000000930D0110930E0108950AE000930D016F
:1006100000930E01022D003039F000911401D2D068
:1006200000930D0110930E0100911501CBD00093A2
:100630000F01103009F41AE0109310010895032DF2
:10064000003069F004E100930D0104E100930E0114
:1006500005E100930F0103E10093100108952ED1ED
:1006600000E100930901DDD208950AE00093100132
:1006700000930F01022D003009F02DD021D00895F4
:100680000AE000930E0100930D01022D003009F0E5
:1006900017D021D00895032D003069F00CE00093AD
:1006A0000D0104E100930E0100E100930F010EE043
:1006B000009310010895002700930901B2D2089514
:1006C00000910B01102F12950F701F7000930D01F8
:1006D00010930E01089500910C01102F12950F70C8
:1006E0001F7000930F01103009F41AE010931001ED
:1006F000089500910B0000930D0100910B000093F1
:100700000E0100910C0000930F0100910A0000936C
:1007100010010895045628F0045638F0045648F0A5
:10072000E8CF1AE01093100107C011E010931001F8
:1007300003C012E0109310010C590A5098F00A50AF
:10074000D0F00A50E0F00A50F0F00A5000F10A50E0
:1007500010F10A5020F10A5030F10A5040F10A50CD
:1007600050F1C7CF1AE020910901243009F410E0BC
:1007700010930F0123C011E010930F011FC012E06E
:1007800010930F011BC013E010930F0117C014E06A
:1007900010930F0113C015E010930F010FC016E066
:1007A00010930F010BC017E010930F0107C018E062
:1007B00010930F0103C019E010930F01065F00931F
:1007C0000E0108950A5068F00A5068F00A5068F067
:1007D0000A5068F00A5068F00A5068F00DE01DE019
:1007E000089510E00AC011E008C012E006C013E04E
:1007F00004C014E002C015E000C0065F0895109127
:100800001001FCD115B95C9A01D210910F01F6D1FB
:100810005C9815B95D9A14D2F9D110910E01EED100
:100820005D9815B95E9AF2D110910D01E7D15E98ED
:1008300015B95F9AEBD15F980895052D003051F4FA
:1008400000910901025030F424D038D00F930BE10D
:10085000502E0F910895F89475D000ED5BD01130B3
:10086000A9F000E057D0113089F0002753D01130A3
:1008700069F000910B014ED0113041F000910C0154
:1008800049D0113019F068D07894089565D07894E3
:100890000895F89457D000ED3DD01130B9F301E040
:1008A00039D0113099F34ED001ED34D0113071F3BD
:1008B0001AD000930B0150D078940895F89442D048
:1008C00000ED28D0113011F302E024D01130F1F204
:1008D00039D001ED1FD01130C9F205D000930C01C1
:1008E0003BD078940895002718E045983FD03ED03B
:1008F000459A3CD008943C98349B8894001F36D08D
:100900001A9599F7459832D03C9A30D0459A2ED016
:100910002DD0089518E0459829D03C98000F08F094
:100920003C9A24D0459A22D021D01A95A1F7459817
:100930001DD03C981BD0459A19D011E0349B11274B
:1009400015D00895459812D044983C980FD0459AF8
:100950000DD03C9A0BD008953C9A459A07D03C980C
:1009600005D0449A3C9A3D9A459A08950F9308E021
:100970000A95F1F70F91089502E00EBF0FEF0DBF3A
:1009800078940FEF04B90AB9002705B90BB900E351
:1009900007B907E608B922243324442455246624E1
:1009A0007724002706BD0093850000938400009300
:1009B0000B0100930C0100930201009303010093CB
:1009C00009010DE000930D0100930E0100930F014A
:1009D0000093100101E000930A0104E005BD03E06B
:1009E0000093810001E000936F0000936E000EE819
:1009F00000937A00B6DFF1D0B6D0CFDC00DF07D0AD
:100A00001CDF25DB18D02CD087D08ED0F6CF0091FC
:100A10000801013279F400910601109107011BD100
:100A200000930201009104011091050114D100937B
:100A30000301D3D008950091000110910301011B1F
:100A400050F00091110110910001101B0091030161
:100A5000011B18F008955A9808955A9A0895089518
:100A600000910A010030D9F34AD00D5000F147D06F
:100A700010911501101BC8F042D010911501101BE8
:100A800009F005C02FD010911401101B70F00091D7
:100A9000010110910201011B28F0062D003019F40C
:100AA00059980895C8D0599A08955998089527D00B
:100AB00010911301011BC8F322D010911301011BE7
:100AC00009F005C00FD010911201011B70F30091C5
:100AD000010110910201011B28F3062D003019F7C6
:100AE0005998089500910B01102F12950F701770EF
:100AF000103021F02AE0020F1A95E9F708950091CD
:100B00000C01102F12950F701370103021F02AE095
:100B1000020F1A95E9F7089500910A01013011F0CA
:100B20005B9808955B9A089500910A01013059F08D
:100B3000E6DF1AE0011739F4D5DF10E0011719F4E8
:100B400001E000930A010895F999FECF11BDF89ACA
:100B500000B50895F999FECFF89411BD00BDFA9A39
:100B6000F99A789408951AE0EFDF009300011BE0F2
:100B7000EBDF009301011CE0E7DF009311011DE0B2
:100B8000E3DF009313011EE0DFDF009312011FE09B
:100B9000DBDF0093150110E1D7DF00931401089506
:100BA0001AE000910001D6DF1BE000910101D2DFC5
:100BB0001CE000911101CEDF1DE000911301CADF9E
:100BC0001EE000911201C6DF1FE000911501C2DF97
:100BD00010E100911401BEDF0895F89400270093FE
:100BE000080100930601009307010093040100939C
:100BF000050107E000937C0078940895E4E3F0E0B9
:100C000020E0E10FF21FC895102D08951F932F9338
:100C100012E328E21A95F1F72A95E1F72F911F9137
:100C200008950F9303E0302E0F9108950F9303E082
:100C3000402E0F9108950F9303E2602E0F910895B7
:100C400000910901003029F4022D003011F02B9899
:100C500008952B9A089526E0169507952A95E1F7B1
:100C60000895002700930A01599A089500270093D8
:100C70000A0159980895EFDDC2DD92DF08959FB70C
:100C80000F931F932F933F93209178003091790019
:100C9000009108010132E1F0039500930801013150
:100CA000E9F0015158F00091060110910701200F61
:100CB000311F20930601309307010AC000910401FF
:100CC00010910501200F311F20930401309305017D
:100CD0003F912F911F910F919FBF189506E00093B0
:100CE0007C00F6CF9FB70F931F932F933F930EEC8B
:100CF00000937A003F912F911F910F919FBF1895FC
:100D00009FB70F931F932F933F93022D003011F045
:100D1000222404C00F9301E0202E0F91032D0030F8
:100D200009F03A94042D003009F04A94052D003062
:100D300009F05A94062D003009F06A943F912F91E2
:0A0D40001F910F919FBF18951895A1
:00000001FF
